:020000040000FA
:060000008AEF2BF0120054
:060008003AEF0AF01200BD
:06002A0006008B570000E8
:100030007E03000004000000875700007A030000E0
:100040000400000065570000890200002200000043
:100050005D57000072030000080000005B570000BD
:100060008203000002000000465700000003000069
:040070001500000077
:100110000401006B040E005D26E20051260DF3CFB2
:1001200001F4F4CF02F4000E0127010E0223F7ECD4
:1001300008F0EF6A14EC0AF0EF9014EC0AF0EF828A
:1001400014EC0AF0EF8414EC0AF0EF9814EC0AF0C7
:10015000EF96F7EC08F0CBEC09F0F7EC08F0E2ECE6
:1001600009F0002BD7D70101986B040E996F9A6B99
:100170009B6B9C6B9D6B12000401006B040E005D79
:1001800036E20051260DF3CF01F4F4CF02F4000E55
:100190000127010E0223EBEC08F0EF50000925E1E6
:1001A000EBEC08F0010EEF6EEBEC08F00B0E9EC1CD
:1001B000EBFF0C0E9FC1EBFFEBEC08F00D0EEB6AB2
:1001C0000E0EEB6AEBEC08F0DBEC09F020EC0AF029
:1001D000EF8020EC0AF0EF96EBEC08F0CBEC09F0A6
:1001E00020EC0AF0EF8200511200002BC7D7FE0C62
:1001F00004010A6B076B040E075D14E20751260D1C
:10020000F3CF08F4F4CF09F4000E0827010E0923F8
:100210009FEC08F0EF50000903E1010E0A6F02D0D5
:10022000072BE9D70A5101E1FE0C0101982B000EC2
:1002300099239FEC08F00B0E98C1EBFF0C0E99C1AF
:10024000EBFF880ED8809855130E995503E2986BF2
:10025000040E996F9FEC08F0A2EC09F0EF909FEC70
:1002600008F00D0EA2C1EBFF0E0EA3C1EBFF9A2BFF
:10027000000E9B239C239D23E6EC09F064EC09F01F
:100280009FEC08F0180E7BEC08F07FEC09F00A0EEA
:10029000E66EE66AA0C1E6FFA1C1E6FF9FEC08F0AA
:1002A000A4EC08F00FEC09F00101020EC66F9FEC00
:1002B00008F0CFEC09F0E6EC09F006EC09F09FEC51
:1002C00008F0D3EC09F09FEC08F0D7EC09F09FECB4
:1002D00008F0F0EC08F09FEC08F0030EEF6EE6EC8F
:1002E00009F084EC09F00401075112000101A45146
:1002F000CFEC08F0EF50040801E0000C010C010104
:10030000A551260DF3CFABF4F4CFACF4000E0401ED
:10031000AB27010EAC23FCEC08F0EF50040806E01C
:10032000ABC4D2F1ACC4D3F1E2EF06F0A5C1AAF19F
:10033000FED80FEC09F00101110EC66FFCEC08F0BD
:10034000CFEC09F0FCEC08F017EC0AF006EC09F031
:10035000FCEC08F0D3EC09F0FCEC08F0D7EC09F069
:10036000FCEC08F0F0EC08F0FCEC08F017EC0AF0FC
:1003700084EC09F0FCEC08F0050EEF6E12000101B0
:10038000A651260DF3CFAFF4F4CFB0F4000E040164
:10039000AF27010EB0239AEC08F00F0EEB50FF08C8
:1003A00001E1000C9AEC08F002EC0AF0020B01E10A
:1003B000000C9AEC08F0100E7BEC08F0EECFC8F1C0
:1003C000EDCFC9F19AEC08F00F0EEB500101C76FA9
:1003D0000101100EC66FCFEC09F09AEC08F017EC93
:1003E0000AF006EC09F09AEC08F0D3EC09F09AEC6C
:1003F00008F0D7EC09F09AEC08F0F0EC08F09AEC71
:1004000008F0100EE9EC09F00D6A0E6A9AEC08F09B
:1004100017EC0AF00B50EE260C50EE220D50EE2297
:100420000E50EE2231EC0AF0EF9231EC0AF0EF9828
:100430009AEC08F03FEC09F09AEC08F0CBEC09F0EC
:1004400031EC0AF0EF82010C0101A751CFEC08F06A
:100450000F0E7BEC08F0EF50FF0802E127EF13F0DE
:10046000A751CFEC08F002EC0AF0020B01E0010EFC
:1004700012000101A851260DF3CFADF4F4CFAEF474
:10048000000E0401AD27010EAE2301EC09F00F0EA2
:10049000EB50FF081EE101EC09F00F0EDFC1EBFF8E
:1004A00001EC09F0EB500101E96FB1EC13F001EC44
:1004B00009F0100EEB6A110EEB6A280E0101FD6FB8
:1004C000FE6B01EC09F00F0EEB500101FC6F47ECE5
:1004D00015F001EC09F0100E7BEC08F0EECFABF458
:1004E000EDCFACF40401CA0EAB5D030EAC5901E3D1
:1004F000000C01EC09F0A2EC09F0EF88A9C1E0F1D1
:100500002EEC13F00401AB2B000EAC2301EC09F030
:10051000100EABC4EBFF110EACC4EBFFCA0EAB5D0B
:10052000030EAC5903E3A8C1A6F129DF010C0101B8
:10053000AA51260DF3CF65F4F4CF66F4000E040142
:100540006527010E662365C4E9FF66C4EAFF2EEC49
:100550000AF001E1000CC0EC13F065C4E9FF66C4C9
:10056000EAFFA2EC09F0EF96010C0101AB51260D58
:10057000F3CF00F4F4CF01F4000E04010027010EC4
:10058000012329EC0AF02EEC0AF01DE029EC0AF018
:1005900002EC0AF0040B08E0280E33EC09F029EC19
:1005A0000AF0A2EC09F0EF9429EC0AF0A2EC09F0B1
:1005B000EF88AEC1E7F1AFC1E8F1ACC1E5F1ADC183
:1005C000E6F181EF13F00B6A0C6A0BC0F3FF0CC06D
:1005D000F4FF12000101B051260DF3CF65F4F4CF02
:1005E00066F4000E04016527010E66232EEC09F067
:1005F0002EEC0AF02DE02EEC09F002EC0AF0040BD0
:1006000008E0280E33EC09F02EEC09F0A2EC09F01A
:10061000EF942EEC09F0120E7BEC08F0EE50ED108A
:1006200008E1C0EC13F02EEC09F0A2EC09F0EF9613
:10063000000C2EEC09F0120E7BEC08F0EE06EF5ADF
:100640007AEC13F0B1C1E9FFB2C1EAFFEF6E010C21
:10065000000C0101B351CFEC08F02EEC0AF001E0E0
:10066000010E120004010F6B006B040E005D01E32C
:10067000EBD00051260DF3CF09F4F4CF0AF4000EAD
:100680000927010E0A2390EC08F02EEC0AF001E095
:10069000D8D090EC08F002EC0AF0100B01E0D1D0B9
:1006A00090EC08F0EF50000901E1CBD090EC08F09D
:1006B000EF50010807E190EC08F002EC0AF0010BA2
:1006C00001E0BFD05FEC2BF004C005F405C006F4D8
:1006D00006C007F407C008F490EC08F01D0E7BEC90
:1006E00008F0EE500401045C016FEE500558026FF3
:1006F000EE500658036FEE500758046F90EC08F068
:10070000210E7BEC08F00151EE5C0251EE580351D2
:10071000EE580451EE5801E394D027EC13F0000991
:1007200001E112005FEC2BF0B3EC08F090EC08F064
:100730001D0E23EC0AF090EC08F0210E7BEC08F083
:1007400084EC09F090EC08F01C0E7BEC08F0EF2A2A
:1007500090EC08F0EF50060A27E0010A25E0020AB3
:100760001CE00F0A1AE00E0A10E0060A05E0010A72
:1007700028E10401020E24D0F2EC09F00B6E030E06
:100780000B5C16E20401120E1BD00401110E0F6F58
:1007900090EC08F0050EEF6E14D0F2EC09F00308AF
:1007A00007E30401010E0CD0F2EC09F0030806E2A5
:1007B00009C4D2F10AC4D3F105DB03D00401100E41
:1007C0000F6F04010F5100083CE2100E0F5D11E0A5
:1007D00090EC08F017EC0AF0EFCF0BF4EE2AEFCF15
:1007E0000CF4EE22EFCF0DF4EE22EFCF0EF4EF2259
:1007F0000CD090EC08F017EC0AF0EECF0BF4EECF33
:100800000CF4EECF0DF4EFCF0EF40FEC09F00FC4A3
:10081000C6F190EC08F0CFEC09F00BC4BEF10CC4AB
:10082000BFF10DC4C0F10EC4C1F190EC08F0D3ECDF
:1008300009F090EC08F0D7EC09F090EC08F0F0EC3F
:1008400008F00401002B11D71200140E0101E76F0C
:10085000E86B0101000EE56F040EE66F81EC13F00A
:100860000101000ED06F040ED16F7FDAB4C1E9FF31
:10087000B5C1EAFF26EC0AF0EECF14F4EECF15F482
:10088000EECF16F4EFCF17F400C218F401C219F43A
:1008900002C21AF403C21BF404011C6B060E1D6F86
:1008A000B6C11EF4B7C11FF4B6C15FF3B7C160F3A0
:1008B0009CEC28F0F3CF1EF4F4CF1FF40C0E0301D0
:1008C000676F686B0301140E656F040E666FD5ECDD
:1008D00028F0F3CF21F4F4CF22F40401211F221FCA
:1008E000240E33EC09F021C4E0F12EEC13F022C405
:1008F000E0F12EEC13F0140E33EC09F0B6C1CAF19E
:10090000B7C1CBF17ED9F3CF21F4F4CF22F40401A7
:100910001051F31802E11151221903E0C0EC13F059
:10092000010C6DEC09F00B6E0C6A140E0B5E000EE0
:100930000C5A0BC023F40B500B6E0C6AE8500101EB
:10094000B65DB66F0C50B759B76F140EB65F000E98
:10095000B75B04016DEC09F00101FA6FFB6B140E3B
:10096000FA27000EFB2334EC15F0B4C1CEF1B5C16B
:10097000CFF10101000ECC6F040ECD6F7AD90401C6
:10098000206FFE0E205D11E2B6C1D9F1B7C1DAF1D8
:100990000101000ED76F040ED86FB4C1D5F1B5C1F7
:1009A000D6F120C4D4F136DA010CC0EC13F0FF0EFE
:1009B0000401205D38E10101B6510401082701015D
:1009C000B75104010923000E0A230B230D51020B1A
:1009D00003E10D51010B05E0082B000E09230A234A
:1009E0000B230FEC09F00101040EC66F04C4C2F121
:1009F00005C4C3F106C4C4F107C4C5F108C4BEF1FF
:100A000009C4BFF10AC4C0F10BC4C1F100C4BCF1F8
:100A100001C4BDF102C4BAF103C4BBF1B4C1B8F161
:100A2000B5C1B9F101D8010C27EC13F00009FCE0C5
:100A3000BAC167F4BBC168F4BCC169F4BDC16AF452
:100A4000BEC16BF4BFC16CF4C0C16DF4C1C16EF422
:100A5000C2C16FF4C3C170F4C4C171F4C5C172F4F2
:100A600004017391739373957397C6C174F4D9ECB1
:100A700013F0F3CF75F4F4CF76F40401000EF35CB9
:100A8000040EF45804E3756B040E766F0DD0360E29
:100A9000D8807555000E765505E2360E755F000E4E
:100AA000765B02D0756B766B776B786B796B7A6B54
:100AB0000101670ED06F040ED16F57D9140E0101DA
:100AC000C827000EC923C6A30ED0040EC827000EE7
:100AD000C9230401020E7B6F040E7C6F7D6F7E6B59
:100AE0007399738B03D004017389739B738D739F08
:100AF00000C27FF401C280F402C281F403C282F416
:100B0000B8C1E9FFB9C1EAFF26EC0AF0EECF83F4E1
:100B1000EECF84F4EECF85F4EFCF86F4876B060E2C
:100B2000886FC8C189F4C9C18AF4C8C15FF3C9C15B
:100B300060F39CEC28F0F3CF89F4F4CF8AF40C0E28
:100B40000301676F686B03017F0E656F040E666FAC
:100B5000D5EC28F0F3CF77F4F4CF78F40401771FC5
:100B6000781F77C465F478C466F4FF0E0101C75D91
:100B700002E1DFC1C7F1140E65DBC8C151F3C9C181
:100B800052F30301060E506FB8C14EF3B9C14FF3D3
:100B900066EC1EF0140E0101E36FE46B0101670EB9
:100BA000E16F040EE26F37EC13F00101C6A30BD026
:100BB000040E0101E36FE46B01017B0EE16F040E93
:100BC000E26F37EC13F0140E3DDBC8C1CAF1C9C1A6
:100BD000CBF117D8F3CF65F4F4CF66F4240E32DBF3
:100BE00066C4E0F12EEC13F065C4E0F12EEC13F0D6
:100BF0000101FD6BFE6BC7C1FCF147EC15F0DCEFAA
:100C000014F00401010E8B6F8C6B8D6B0101CAC156
:100C10000BF0CBC10CF0CA07000ECB5B0B500C10D5
:100C200020E07AEC13F004018E6F8B510AE18E51B3
:100C30008C258C6F8E518C5D0DE28D2B0BE18C2BF6
:100C400009D08E518D258D6F8E518D5D03E28C2BD9
:100C500001E18D2B8B5102E0000E01D0010E8B6F54
:100C6000D5D704018D1D8D6F8C1DF36E8DC4F4FFDF
:100C700012000401FE0E276F266B040E265D44E26F
:100C8000265118DB87DAEF5000093BE083DA0B0EC0
:100C9000A0DB3FDB020E2FDA41DB33E10E500C18F4
:100CA00030E178DAEF50010802E126C427F472DA65
:100CB0000D0E8FDB2EDB32DB24E10E500C1821E110
:100CC000CEC1E9FFCFC1EAFFC1DBEECF0FF0EECF1F
:100CD00010F0EECF11F0EFCF12F05CDAEE52B6DB8F
:100CE000EE5000010F190DE1EE5010190AE1EE501F
:100CF000111907E1EE50121904E103E10401265134
:100D000012000401262BB9D72751D4DAFE0E275D35
:100D100027E040DAEF50010823E10A0EE66EE66AAA
:100D2000CEC1E6FFCFC1E6FF35DA0EDAF550F1DAD3
:100D3000020E4FDB2FDA0B0E0BC0EBFF0C0E0CC0BC
:100D4000EBFFE7DA86DA26DAF0DA24DAFBDAEF9676
:100D500021DA21DB1FDAF6DAEF82040127511200D3
:100D6000FE0E275D01E1FF0CFE0C4FDBCDD9F3CF6A
:100D7000EEFF0CC0EDFF49DB020E2EDB020EF3CFBF
:100D8000EBFF030E82DA040EF8DA040E18DB080E0D
:100D9000F4DA080E14DB0E0E1FDB0E0EF3CFEBFFA2
:100DA0000F0E73DA100E18DB100EF3CFEBFF110EDF
:100DB0006CDA120E11DB120EF3CFEBFF130E0CC028
:100DC000EBFF1200E2D90F0EEB50FF0806E0DDD971
:100DD00056DADBD9E0DA48DBEF82D7D9ECDAD5D9BD
:100DE0000D0EEB6A0E0EEB6AD0D938DB02E0C0ECD8
:100DF00013F03ADBEF96C9D9E5DA36DBEF98C5D9BF
:100E000001DB010B04E0C1D9010EEF6E1200BDD968
:100E1000EF6A12000401366B0101D451260DF3CFA5
:100E200034F4F4CF35F4000E04013427010E3523D9
:100E300091DAEECF2CF4EECF2DF4EECF2EF4EFCFEF
:100E40002FF48CDAEECF30F4EECF31F4EECF32F473
:100E5000EFCF33F46AD9040E4ED948DA0101D951E3
:100E6000040124270101DA5104012523000E262361
:100E70002723D0DA76DAA6DAB2DA01083AE1C0EC52
:100E800013F001019A2B000E9B239C239D2366DA0D
:100E90001BDA0401242B252326232723CBDABADAF5
:100EA0005DDA32DA52DA020B14E00A0EE66EE66A16
:100EB000D5C1E6FFD6C1E6FF22D946D9F55035D9CE
:100EC000C8D91DD932DA0401120E366F18D9020EB4
:100ED000E2D0040E366F24C428F425C429F426C4B5
:100EE0002AF427C42BF421D906D900DA08D963DA09
:100EF000DFD02BDA040B04E0C0EC13F09CEF09F018
:100F000014D9080EF8D804012851EE1801E0CED00B
:100F10002951EE1801E0CAD02A51EE1801E0C6D0DE
:100F20002B51EE1801E0C2D001E0C0D058DA02081F
:100F30000AE183DA01E1BAD07DDA13DA040EEF6E4A
:100F4000A8D92CE3B3D04BDA03082AE1FED9020B6F
:100F500001E1ACD0242B000E2523262327236ADAB7
:100F60006CDA06E0100E366FCAD8040EEF6E13D09E
:100F7000120E366FC4D8020EEF6E282B000E2923F6
:100F80002A232B23EBD928C4EEFF29C4EEFF2AC461
:100F9000EEFF2BC4EEFF7DD901E388D027DA88D09D
:100FA000C4D8040EA8D8EECF0BF0EECF0CF0EECFE5
:100FB0000DF0EFCF0EF0CED90B50EE1808E10C502B
:100FC000EE1805E10D50EE1802E10E50EE1802E0A9
:100FD000C0EF13F02FDA03DA040844E12EDA0BE055
:100FE0008ED80F0EEB50FF0806E089D848D987D875
:100FF000D2D93DDAEF82A9D9010B15E00401110E17
:10100000366FACD9EFCF28F4EE2AEFCF29F4EE22D9
:10101000EFCF2AF4EE22EFCF2BF4EF229BD905D9A4
:101020006ED80A0EEF6E35D941E269D817DA05E1BC
:10103000DDD90401100E366F3BD00401366B8ED91A
:1010400030C4EEFF31C4EEFF32C4EEFF33C4EEFF16
:1010500081D92CC4EEFF2DC4EEFF2EC4EEFF2FC4A9
:10106000EEFF24D0BCD90A0805E1C0EC13F0E5D9A5
:101070001FE01AD0B4D9050810E1C0EC13F065D90F
:10108000010B16E00401100E366F64D9CED8D5D905
:101090000BE135D8060EEF6E0BD0A1D9060808E19A
:1010A000C0EC13F0CAD904E047D902D0C0EC13F069
:1010B0000401365100081EE2B2D836C4C6F124C479
:1010C000C2F125C4C3F126C4C4F127C4C5F128C4A4
:1010D000BEF129C4BFF12AC4C0F12BC4C1F125D887
:1010E000DFD823D8020E07D8E0D8D5C1B8F1D6C1D1
:1010F000B9F19ADC1200E926000EEA22120034C48B
:10110000E9FF35C4EAFF1200EECF5FF3EDCF60F3E5
:101110009CEC28F0F3CF0BF0F4CF0CF005EF0AF0C5
:1011200009C4E9FF0AC4EAFF1200D7C1E9FFD8C128
:10113000EAFF1200AFC4E9FFB0C4EAFF120008C41E
:10114000E9FF09C4EAFF1200EE52E9CF0BF0EACF43
:101150000CF0E9CFE6FFEACFE6FFD2EC27F0F56E20
:10116000060EE15E120004C00BF005C00CF006C0D4
:101170000DF007C00EF0120004C0EEFF0CC0EEFF31
:101180000DC0EEFF0EC0EEFF1200D2C1E9FFD3C1C9
:10119000EAFF120024C4E9FF25C4EAFF1200260D6D
:1011A000F3CFE9FFF4CFEAFF000EE926010EEA22B1
:1011B0001200EECFC2F1EECFC3F1EECFC4F1EFCF0C
:1011C000C5F1120024C4EEFF25C4EEFF26C4EEFFD5
:1011D00027C4EEFF120001C4E9FF02C4EAFF1200B7
:1011E000EE52E9CFB8F1EACFB9F114EF05F001C43E
:1011F000E9FF02C4EAFF1200ABC4E9FFACC4EAFF96
:101200001200ADC4E9FFAEC4EAFF1200EECFBEF19A
:10121000EECFBFF1EECFC0F1EFCFC1F1120001016F
:10122000C86BC96B0101C7691200EF2AEECF24F425
:10123000EF22EECF25F4EF22EECF26F4EF22EFCF10
:1012400027F412000101FD6FFE6BC7C1FCF147EFEF
:1012500015F0EECF0BF0EFCF0CF0120065C4E9FFF4
:1012600066C4EAFF12000101FA6FFB6B34EF15F060
:10127000700EEE6E170EEE6EEE6AEE6A12000F0E34
:10128000EB500101EA6FB7EF13F00CC0EBFF05EF75
:101290000AF00101000ED880D955000EDA5512006F
:1012A000EECFBCF1EDCFBDF11200EECFBAF1EDCF34
:1012B000BBF11200260DF3CF24F4F4CF25F4000E79
:1012C0002427010E252312009AC1EEFF9BC1EEFFD9
:1012D0009CC1EEFF9DC1EEFF12000C51F00BE842E5
:1012E000E842E842E842040DF3501200EECF24F445
:1012F000EECF25F4EECF26F4EFCF27F41200EE6AFE
:10130000EE6AEE6AEE6A1200EE2AEE22EE22EE227B
:101310001200CCC1E9FFCDC1EAFF1200EECF0DF003
:10132000EFCF0EF00D500B1812000D0E0BC0EBFF9F
:101330000E0E0CC0EBFF120034C4D2F135C4D3F151
:10134000E2EF06F0250E7BEF08F0EFDE0D0ED3DEA8
:10135000EF501200D4DE180E7BEF08F0D0DE17EF4E
:101360000AF0CDDE1C0EC7DEEF6A5FEC2BF0FBDE71
:10137000C6DE1D0E68D87FEF08F0BDDEEECF61F34C
:10138000EECF62F3EECF63F3EFCF64F3A1EC28F07E
:10139000EADE05EF0AF00F0EAEDEEF681200180E5F
:1013A000AADED9EF08F00D0EA6DE50EF09F00B0E05
:1013B000A2DE55EF09F0EE5249D87FEF09F043D88D
:1013C00005EF0AF0210E97DE38EF09F0B8DE17EFCF
:1013D0000AF091DE29EF09F08EDE84EF08F08FDE4F
:1013E000EF5012009DDE1C0EEB50120040D8EF862D
:1013F00086DE120ED9C1EBFF130EDAC1EBFF37D830
:10140000EF8412009FDFEF501200D0C1E9FFD1C17D
:10141000EAFF1200A3DFEECF28F4EECF29F4EECFDF
:101420002AF4EFCF2BF41200E2DEA2EF09F0140E43
:101430007BEF08F08FDFE2EF08F087DF100B120080
:10144000CADEA2EF09F057DEBCEF08F0060E7BEF14
:1014500008F000C4E9FF01C4EAFF1200D3DF080B63
:10146000120068DEA2EF09F090DEA2EF09F047DE7D
:04147000A2EF09F0EE
:0C147400DACFE4FFE2CFDAFFE9CFE4FFBB
:10148000EACFE4FF00EE0BF0080EE80403E3EECF32
:10149000E4FFFBD7E6526DEC2BF0E55200EE12F0C4
:1014A000080EE80403E3E5CFEDFFFBD7E5CFEAFF45
:1014B000E5CFE9FFE5CFDAFF1100ACA2FED71DC2F0
:1014C000ADFF120002011EC2E9FF1FC2EAFF1E2B80
:1014D000000E1F23EFCF08F4EF5004E008C41DF204
:1014E000ECDFF0D7120061D956EC2BF06EEC21F056
:1014F0007CD981BA0AD098EC0EF002017D0EFC6F07
:101500004D0EFD6FC2EC29F0EDDAA6EC25F008ECEB
:101510000FF032EC1BF0020118A10AD098EC0EF08B
:1015200002016C0EFC6F4D0EFD6FC2EC29F006D06F
:101530000301010E006F0301070E7A6F5FEC2BF0C1
:1015400003010151045C0B6E025105580C6E0351EE
:1015500006580D6E04519DEC0EF00BE35FEC2BF082
:1015600004C001F305C002F306C003F307C004F38F
:101570008978B1EC25F020EC0FF041EC1BF04FD84E
:101580000301005103017D5DD9E00201010E226FCC
:101590000201000E206F020E216F17D87DC300F3E9
:1015A000020118A1CBD70201CE0EF96F89EC29F008
:1015B0000A0E0301005D02E2300E01D0410E00254B
:1015C0000201FE6FD4EC29F0B9D70201225108E0E4
:1015D000AFDB02018C0EFC6F4D0EFD6FC2EC29F0EB
:1015E000A7DB85DB4FDB02E067DB01D06BDB7FDB5A
:1015F000010EF5EC0EF002E05FDB01D063DB77DB80
:10160000020EF5EC0EF002E057DB01D05BDB6FDB86
:10161000030EEBDB02E0FAEF0EF001EF0FF0810EAC
:10162000C26E0401640E006F005100070009FCE166
:10163000C284C2B4FED7C3CF00F4C4CF01F4230EDA
:10164000E66E020E6EDB840EC16E890EC26E040160
:10165000640E006F005100070009FCE1C284C2B4AF
:10166000FED7C3CF00F4C4CF01F42B0EE66E020EFA
:1016700058DB8E0EC16E120033C2E9FF34C2EAFF9E
:101680008EDB0401656FE850010A23E0010A1AE1CC
:10169000020E0201EA6A3325E96E3451EA227FDB49
:1016A0000401666FE850010A04E0010A03E189764B
:1016B00001D089740D0EE66EE66A9D0E0B6E4D0E1E
:1016C00067EF0EF00A0EE66EE66AAA0E0B6E4D0E7E
:1016D000FEDA120002013651040A3AE0070A1FE05E
:1016E000010A0BE0030A05E0010A3CE189B603D0D8
:1016F00031D089A42FD0300E30D03751381102E1CB
:10170000376B386B3751EA6A230FE96E020E2BDB19
:10171000230FE96E020EEA22EF5024E011D0375178
:10172000381102E1376B386B3751EA6A2B0FE96EDB
:10173000020E19DB2B0FE96E020EEA22EF5012E0C7
:10174000372B000E382337C2F3FF38C2F4FF1200E4
:1017500081AA02D0310E01D0300E39C2E9FF3AC25F
:10176000EAFFEF6E0B680C680BC0F3FF0CC0F4FFD0
:101770001200030EE66EE66AB40E0B6E4D0E23DB0E
:101780003BC2E6FF3CC2E6FF02DB0EE1090EE66E5D
:10179000E66AB80E0B6E4D0E16DB3DC2E6FF3EC28A
:1017A000E6FFF5DA01E1010C000C8E0EC16E030EAE
:1017B000926E809A89848986F19E5FEC29F00201FD
:1017C000800EF96F89EC29F002015C0EFC6F4D0E62
:1017D000FD6FC2EC29F0200EAC6E900EAB6E0F0EBA
:1017E000AF6ED56AF28EF28C120002010A0E006F03
:1017F000016F050E026F0F0E036F0A690B690C690A
:101800000D6B0A0E0E6F0F6F050E106F0F0E116F1E
:10181000046B040E056FA30E066F076B086B096B54
:1018200018810401000E046F020E056F03012B6B7B
:10183000BDDA1DEC24F00401036F26EC24F0550EF4
:101840000401035D1BE1010E03012B6FAFDA0401FC
:10185000036B0351B1DA10E21DEC24F0E66E0401D3
:1018600004C4E9FF05C4EAFF042B000E0523E5527A
:10187000E750EF6E032BEDD726EF24F040EF0CF08E
:101880000401000E016F020E026F0301286B296B29
:101890000301A00E276F9CEC23F00301550E2D6F62
:1018A000FFEC23F00401006B005186DA0EE201C464
:1018B000E9FF02C4EAFF012B000E0223EFCF2DF354
:1018C000FFEC23F00401002BEFD713EF24F002010B
:1018D0003FC2F6FF40C2F7FF3F2B000E4023080037
:1018E000F5CF00F4F55004E000C41DF2E6DDEFD7BB
:1018F00012000401016B9EAAFED7AECF00F40D0EBC
:101900000401005D17E00A0E005D14E0012B0201E6
:1019100041C2E9FF42C2EAFF412B000E422300C44C
:10192000EFFF41C2E9FF42C2EAFFEF6A43514307BA
:101930000009E1E104010151120044C201F445C271
:1019400002F40401036B44C2E9FF45C2EAFFEFCF92
:1019500000F4EF5021E02E0E0401005D11E10201C0
:1019600044C2E9FF45C2EAFF442B000E4523EF6A5B
:10197000C7D9032B02DA44C201F445C202F407D0EE
:10198000300E005D03E30051390801E2000C020152
:10199000442B000E4523D7D7B3D9EFD9030E04014A
:1019A000035D01E0000C010C9EAAFED7AECF00F44F
:1019B000310E0401005D05E3390E005D02E20051C5
:1019C0001200390C02010D0E0DDA02010A0E0ADABC
:1019D000300E0201485DFF0FE96EEA6AD890E936E1
:1019E000EA36050EE926030EEA22EECF3FF2EDCFEE
:1019F00040F26DDF02014851380A72E00F0A6EE0D2
:101A0000010A6AE0030A66E0010A34E0070A2DE0F1
:101A1000010A26E0030A01E012008F0EE66E040EB2
:101A2000E66E12C2E6FF13C2E6FFD5D902018F0EA1
:101A30001E6F040E1F6F46DD2CD9000935E08F0E96
:101A4000E66E040EE66E82EC22F0E552E552F3CF2C
:101A500012F2F4CF13F2F4CF08F2F3CF09F212002E
:101A60000401000EA76F020E09D004010E0EA76F2D
:101A7000020E04D004010A0EA76F020EA86F020125
:101A8000226BA7C420F2E8CF21F29FDD02D9020128
:101A9000A30E466F040E476F02018F0E446F040EB3
:101AA000456F4BDF000909E102011B0E3F6F4F0E2E
:101AB000406F0DDF9EBA0DD0FDD7A7C4E9FFA8C4C3
:101AC000EAFFA3C4EEFFA4C4EEFFA5C4EEFFA6C4C4
:101AD000EEFF1200188112001891120086EF0DF02F
:101AE00040EF0CF00201C20E3F6F4D0E406FEFDE73
:101AF0005BDF0401AB6F390EAB5D03E0ABC448F2B2
:101B000061DF380E0401AB5DEDE112000401006BF2
:101B1000046B10EC22F0F3CF02F4F4CF03F418D9E5
:101B20006DEC2BF05FEC2BF004C08BF405C08CF453
:101B300006C08DF407C08EF4870EE96E040EEA6EBF
:101B4000EE500401045C0B6EEE5005580C6EEE5026
:101B500006580D6EEE50F1D805E3FAD80201150EC5
:101B600041D989749EAADCD70401045101E075D0E3
:101B70006DEC2BF09EAAF8D78974AECF01F4040166
:101B80000051030A21E0010A1CE0030A15E00105E7
:101B900002E1010E17D0040E015D0AE18984E5EC33
:101BA00021F00201060E1ED90401010E046FDCD7DC
:101BB0000201150E17D9D8D7060E066F056B020E57
:101BC00001D0030E006FD0D70551052BEA6A070F2D
:101BD000E96E040EEA2201C4EFFF05510B6E0C6A98
:101BE0000C50000AE8AE02D00C3405D0800ED8802C
:101BF0000B54000E0C54B8E202C441F303C442F388
:101C000018EC22F00401060E066F016B01510B6EF9
:101C10000C6A0C50000AE8AE02D0D89004D0800EB6
:101C20000B5C000E0C580DE20151EA6A070FE96ED9
:101C3000040EEA22EFCF43F32EEC22F00401012B35
:101C4000E5D748EC22F0F3CF02F4F4CF03F406C456
:101C50001DF233DC0401006B87D7010C4B0EE66EDE
:101C60007AEC2BF0E5521200140EE66E7AEC2BF0B3
:101C7000E5521200F29E050EE66E98EC2BF0E5524E
:101C8000F28E1200EF50E66EE66AA5D802012251EC
:101C900012000201290EA6D802013A0EA3D80201B1
:101CA000200EA0D80201140E436F02018F0E416F67
:101CB000040E426F79EF0CF09DD802012E0EFE6FDC
:101CC000D4EF29F09ED802012E0EF2EF0EF07BD851
:101CD00033C2E9FF34C2EAFFEECFE6FFEFCFE6FF03
:101CE000FDEC27F0F56E070EE15EF5501200000ED8
:101CF000E66E040EE66E20C2E9FF21C2EAFF120082
:101D000001C4E6FF02C4E6FF82EC22F0E552E55290
:101D1000F350E66E46C20BF047C20CF004010351CB
:101D20001200E66E00C4E6FF01C4E6FFEBEF0EF022
:101D30000201C00EF96F89EF29F007580E6E320EBE
:101D40000B5C000E0C58000E0D58000E0E581200C1
:101D50005FEC2BF004C087F405C088F406C089F45A
:101D600007C08AF41200EA22EF5039C2E9FF3AC2F2
:101D7000EAFFEF6E3751EA6A12000F010B24E96F98
:101D8000000E0C20EA6FE552E750EF6E1200B3EC44
:101D900027F0F56E070EE15EF55000091200EE50D7
:101DA000EFCFEAFFE96EEF50D00F12002C6B03016A
:101DB000A00E2A6FD2EF23F00B6E0C6A1D0E0B5C87
:101DC000000E0C5812000C6E0D6A0BC0E6FFE66E9A
:101DD0000DC0E6FF1200F7EC22F0E552E552E552A5
:101DE000E55212001D6F5DEF0AF0E926000EEA22AF
:101DF00042EF0EF00201000EFA6F040EFB6FB1EF1E
:101E000029F00201000E1E6F040E1F6F62EF0AF030
:101E10000401036B020E035D12E2500E01019E6F7E
:101E20009F6BBCEC00F0E66E04011DDBE552E75051
:101E3000EF6E19DB030EECDAEF6A032BEBD712001F
:101E40000401B36B020EB35D06E2B3C4BFF204D863
:101E50000401B32BF7D712000201BF510A0DF3CFD3
:101E600061F4F4CF62F4AB0E04016127020E622329
:101E7000010E546F0401545101E12AD1546BBEDAB2
:101E80000DDB03E12FDBEF6A1200B8DA030EEB5033
:101E9000090A01E10CD1080A01E1F8D00A0A01E1BE
:101EA000A6D0090A01E185D0020AE4E1A7DAFDDA49
:101EB000E1E00401010E546F526B536B0401500EAC
:101EC000525D000E535914E252C4B1F153C4B2F141
:101ED000522B000E5323000E0101B127040EB22332
:101EE0008DDAEF500101B06FEAEC02F00009E6E193
:101EF000000E04015225E96E040E5321EA6EEF6ACA
:101F000002DBF0DA020EEF6E0401050E5F6F76DA87
:101F1000090E7EDAE9CFC8F2EACFC9F202015F0EFC
:101F2000C66F040EC76F0201550EC46F040EC56F55
:101F30000201000EC26F040EC36F6BD90401516F12
:101F4000E85098E15F5101080EE25FC435F20201EA
:101F5000550E336F040E346F3CEC0BF04FDA090E64
:101F600057DA030EEF6E55C43DF356C43EF377ECDB
:101F700021F0A9DA43DAA0DA41DAEE52FF0EEE18C8
:101F80000AE1FF0EED1807E139DA080E41DAEF6ACF
:101F900035DA030E08D032DAEE52EE50ED1006E1DB
:101FA0002DDA080EB6DA34DA020E90D09BDA0B0E78
:101FB0008DD0BFDA01E15ED721DA080EEB50E96E71
:101FC000EA6AD890E936EA36720EE926030EEA226A
:101FD000EECF63F4EDCF64F439DA02E09FDAFCD798
:101FE0000DDAEF500101A66FBFEC01F05DD0A1DA70
:101FF00001E140D70401010E546F606B60510B6E1C
:102000000C6A1F0E0B5C000E0C5807E26051F76A59
:10201000DA0FF66E550E6EDAF1D7F0D9090EEB50E5
:10202000140DF3CFF6FFF4CFF7FF4E0EF626550E44
:10203000F722F6CF63F4F7CF64F408DA02E06EDA41
:10204000FCD7606B60510B6E0C6A040E0B5C000ECB
:102050000C5807E26051F76AFA0FF66E550E4ADA2D
:10206000F1D7CCD9090EEB50030806E1C7D9070E0A
:10207000CFD9010EEF6E04D0C1D9070EC9D9EF6ACE
:10208000BDD9040E46DAC4D9010E20D0B7D90DDA75
:1020900001E039DA61C4C0F262C4C1F21AD80009A1
:1020A00001E1E8D6E5EC21F01DDA090E0FD0A6D942
:1020B000F5D901E1DFD63DDA01E1DCD69FD9EF5059
:1020C0000101A56F7FEC01F00DDA0A0EEF6ED2D69A
:1020D000120099D9EE52EECF3FF3EDCF40F3ECEC86
:1020E00021F091D9A2D901E18ED00401B16B8BD935
:1020F000040EEB50080812E0FDEC21F00401B26F71
:102100000301381D0BE1391D09E10DEC22F07BD9EB
:10211000EF500101A66FBFEC01F0010C74D9070E5E
:10212000EB5000096BE06FD9040EEB50080A37E062
:102130000E0A23E0030A0CE0060A5CE1250E040106
:10214000B25D03E1D3D9050E53D0010EB16F53D068
:10215000250E0401B25D03E1010EB16F47D0300ED0
:10216000B25D100DF350E66E4ED9080E51D9E5520E
:10217000E750EF6EBBD9060E3BD0300E0401B25DC6
:102180000B6E41D9080E44D90B50EF12AFD9080E8F
:10219000EF6E39D9050EEB6A060EEB6A2CD0020100
:1021A000B20E396F040E3A6F2ED9050E31D9EECF2B
:1021B00037F2EDCF38F227D9080EEB500201366F17
:1021C0006AEC0BF080D91FD9050EF3CFEBFF060E9A
:1021D0000CC0EBFF0401010EB16F15D9050E18D923
:1021E000FF0EEE1808E1FF0EED1805E17FD9030E92
:1021F000EF6E01D0FFD7B15101E173D7B2C4A9F19D
:1022000002D91AD96ED70DEC22F05DD9FCD854D979
:10221000000C0401666B686B696B656B030EE66E00
:10222000E66AFF0E0B6E550E31D9C2C2E6FFC3C27D
:10223000E6FF24D908E1040E0201C227000EC323E1
:102240000401676B01D0020CFCD8EF50200802E1BA
:102250003FD9FAD771D9200E04016A5D5EE06A5158
:102260005CE00D0E6A5D59E00A0E6A5D56E0C6C27A
:10227000E9FFC7C2EAFFEF50655D4FE26651020A0F
:1022800015E0030A0DE0010A46E165514CD954D925
:102290002F0E04016A5D28E05C0E6A5D3CE124D0EB
:1022A0006551652B40D90401020E666F45D93F0E7A
:1022B0006A5D18E0260E6A5D15E02B0E6A5D04E18A
:1022C000200EBFD8EF6E27D02E0E6A5D08E165059F
:1022D00006E1FED8C2C268F4C3C269F41CD03D0E48
:1022E0006A5D05E1AED8EF6A010E666F14D02F0E5D
:1022F0006A5D03E05C0E6A5D0EE1010E02010C6A8C
:10230000C2250B6EC3510C220401650585D80BC094
:10231000EEFF0CC0EDFFDCD89DD793D8EF6A070E17
:10232000DCD8EF6E6851691139E068C4E6FF69C412
:10233000E6FF87EC28F0E552E552F3CF68F4F4CFDE
:1023400069F40401320E6B6F550E6C6F6A6B6A5143
:102350000B6E0C6A070E0B5C000E0C581FE2030E8E
:10236000E66EE66A6BC40BF06CC40CF00D6A6BC4CD
:10237000E6FF6CC4E6FF0DC0E6FF68C4E6FF69C473
:10238000E6FF7CD804E1A9D86AC4EFFF07D0040EA9
:1023900004016B27000E6C236A2BD9D70401655109
:1023A00025E1090EE66EE66A030E0B6E560E6ED838
:1023B000C4C2E9FFC5C2EAFFEECFE6FFEFCFE6FFFA
:1023C000FDEC27F0F56E070EE15EF550C4C2E9FFA3
:1023D000C5C2EAFFEE50EFCFEAFFE96E090E18D84A
:1023E000EF6A010E7AD8EF6E0401652BC6C2E9FFD1
:1023F000C7C2EAFF65C4EFFF6751120061C4E9FF7D
:1024000062C4EAFF1200C0C2E9FFC1C2EAFF1200C3
:10241000E926000EEA221200020D0201C451F32443
:10242000E96EC551F420EA6E1200EF500101A76F6A
:1024300024EC02F000091200EF500101A86F39EFFF
:1024400002F0C2C2E9FFC3C2EAFF1200040163C482
:10245000F6FF64C4F7FF632B000E64230800F5CF7A
:1024600060F4F550120003510A0DF3CFE9FFF4CFE9
:10247000EAFFAB0EE926020EEA221200B3EC27F0C7
:10248000F56E070EE15EF550000912000C6E0D6A44
:102490000BC0E6FFE66E0DC0E6FF1200EF50010133
:1024A000A46F76EC01F000091200EF500101B36F48
:1024B00029EC03F000091200010EF3CFEBFF020E2E
:1024C0000CC0EBFF1200F3CF0BF0F4CF0CF01200B6
:1024D0000201C22B000EC3231200C8C2E9FFC9C209
:1024E000EAFF12008BDF030E08EF12F08CDF040E00
:1024F00008EF12F0F7220800F5CFA9F17FDF9CDF8B
:102500000401602B12007ADFEF500101AA6F97EFF0
:1025100002F07EDF030EEF6EFEEF11F060C4A9F152
:102520006DDF1CEF12F078DFC2C2EEFFC3C2EDFF19
:10253000120064DF15EF12F084DFEFCF6AF41200AF
:102540000401006B0051E5DA15E20051040DF3CFF0
:102550000BF0F4CF0CF0400E0B26000E0C220051B5
:10256000B8DA0BC0EFFF0051B4DAEE52010EEF6E95
:10257000002BE8D70101DF6B32DAC5DA01011F0E4B
:10258000EFDA0101F56F01011F0EB2DABCDAB3DA3E
:10259000800B5CE00101210EA6DAB5DA0101480EDC
:1025A000F56F01010E0EF7DAC0DA040EF56F0101C6
:1025B0000C0EE8DAD8DAC3DA440EF56F0101010E29
:1025C000E1DA5F0EF56F0101020EDCDA5E0EF56FE7
:1025D000D5DAC0DA0F0ED6DA610E85DA04C2F5F16B
:1025E0000101010E85DA05C2F5F10101020E80DA62
:1025F00006C2F5F1C3DA07C2F5F10101040E78DA7B
:1026000008C2F5F10101050E73DA09C2F5F1010105
:10261000060E6EDA0401006B080E005D0AE201018D
:10262000F569080E04010025010162DA0401002B9E
:10263000F3D70101440E7EDA0101440EDD6F010182
:10264000220E51DA5CDA0D0EF46FD9D912000101B5
:10265000F66BE0D9040B01E0000C010C96DA120EC7
:1026600042DAE0C1F5F10101100E78EF15F0010E2C
:102670000101E3150B6E0C6AE3510B240401A26FF8
:102680000101E4510C200401A36F88DAA2C4F5F122
:1026900001010A0E2DDAA3C4F5F101010B0E72DA65
:1026A000120EF56F0101F46BAAD90101E3C10BF021
:1026B000E4C10CF0E307000EE45B32DA0DE2E1C1A5
:1026C000E9FFE2C1EAFFE12B000EE223EFCFF5F1D3
:1026D0000101100EF46FE8D7E369E46BE351E411F4
:1026E00008E009DA400B05E10101E307000EE45BB5
:1026F000F5D712004ADA0A0EF6D90101100EB0EF32
:1027000015F0E7C131F4E8C132F448DA31C4F5F12B
:1027100001010A0EEDD932C4F5F101010B0E32DAD6
:102720000A0EE1D90101E7C10BF0E8C10CF0E7079F
:10273000000EE85BF5D910E20101100E11DAE66E29
:102740000101E5C1E9FFE6C1EAFFE52B000EE62342
:10275000E552E750EF6EE6D731C4F3FF32C4F4FF21
:1027600012000101E951B5D9EE52EF6A12000101E0
:10277000EA51AFD9EE52010EEF6EEAC1DFF112005D
:102780000101DD050401676FE8500B6E0C6A0C5007
:10279000000AE8AE02D0D89004D0440E0B5C000EC4
:1027A0000C5802E25E0E676FD1D967C4F5F1BEEF37
:1027B00015F0DFD904018B6FC9D90101DE51040185
:1027C0008B5D07E25F0E0101D880DE5504018B2589
:1027D00004D00101DE5104018B5D8C6FE8500B6E5B
:1027E0000C6A1B0ED8800B56000E0C560BC08CF4D6
:1027F0000BC08EF48D6B8DC4F3FF0BC0F4FF120081
:102800000101E00E70D90101030EAAD90401006F85
:102810009DD904010051040B01E0000C010CEDC135
:10282000E9FFEEC1EAFFEF6866D9100B0FE0010186
:10283000210E59D90101F96909D961D976D993D9FC
:1028400085D99EDF87D90D0E53D9000C92D904018A
:10285000126F7CD90101DD510401125D58E0DDC128
:1028600014F4136B13C4F7F1DDC1F8F1DFD8120EC5
:102870000101E76FE86B0101000EE56F040EE66FE2
:1028800040DF04010051010B3DE0400E025D000EEF
:10289000035938E3EE0ED8800255050E035532E396
:1028A00010C45FF311C460F39CEC28F0F3CF10F474
:1028B000F4CF11F4060EE66EE66A0A0EE66E040E1A
:1028C000E66EEBC1E9FFECC1EAFFEBC10BF0ECC136
:1028D0000CF0EBC1E6FFECC1E6FFD2EC27F0F56EA1
:1028E000060EE15EF550080E0401115D0BE110517A
:1028F00003E0060E105D06E1EDC1E9FFEEC1EAFF5F
:1029000010C4EFFFDDC1DEF101C4DDF1010C000CEC
:1029100001010A0E0FD946D9EFCFA0F404019F6B35
:102920009FC4F7F1A0C4F8F181D8060E0101E36F4E
:10293000E46BEFC1E1F1F0C1E2F199DE04C2E0F134
:102940008DDE05C2E0F18ADE06C2E0F187DE07C255
:10295000E0F184DE08C2E0F181DE09C2E0F17EDE52
:102960000101F15103E10401A16B03D00401060E42
:10297000A16F0101080EE06F71DEA1C4E0F16EDE0F
:102980000E0E0101F227000EF3233C0EF25D000E45
:10299000F35903E2400EF26FF36BF2C19FF4F3C1FF
:1029A000A0F4F2C1F5F10101050EA2D8A0C4F5F121
:1029B0000101060E78EF15F0C2D8240E94D8040158
:1029C0008B6B8B51A6D80AE28B5183D8EE52EF5015
:1029D00003E08BC4DFF112008B2BF3D71200956854
:1029E000816AE00E936EF19E848284808484966A6C
:1029F000050EE66E98EC2BF0E55284941200F4C1BB
:102A000081FFE00E936EF5C183FF956A8492848204
:102A1000956812009568F6C181FFE00E936E849070
:102A200083CFA4F484800401A4511200F7C1A2F45E
:102A3000F8C1A3F4B3D8A2C4F5F10101080E58D827
:102A4000A3C4F5F10101090E78EF15F0F9C116F4F0
:102A50000401156B15C40BF016C40CF01507000E1D
:102A6000165B5ED8F7E31200DEC168F40401120EB3
:102A7000676F0101FA51040167270101FB5104014D
:102A8000682367C4F7F168C4F8F116EF15F0FCC1CC
:102A9000DFF188D8EFCF8CF404010E0E8B6F0101AB
:102AA000FD5104018B270101FE5104018C238BC4CD
:102AB000F7F18CC4F8F116EF15F00101090E50D8AA
:102AC0000401016F0101080E4BD8F36E01C4F4FF3D
:102AD0001200E96EEA6AD890E936EA36DB0EE9269A
:102AE000010EEA221200F56F0101F46BFFEF14F002
:102AF000F46FFFEF14F00101070EB0EF15F00101C4
:102B0000F56B010112000A0EE66E7AEC2BF0E5522D
:102B100012000B6E0C6A010E0B5C000E0C581200BA
:102B2000D8800B54000E0C5412000A0E34D80B0E31
:102B3000C2EF15F0F56F0101070E78EF15F032D8EE
:102B4000EFCFF5F10101040EC2EF15F00101200EE7
:102B500073EF15F00101F5690101070ECBEF15F0D8
:102B6000F66F0AEF15F0020EF56F01010D0E78EF0A
:102B700015F00101600EB7DF7BEF15F00101030EC8
:102B800078EF15F0B5DF010112000101010EF56FBC
:102B9000010195EF15F0ACDF7FEF15F00101400E5C
:0C2BA0009AEF15F00101DF5169EF15F00C
:042BAC00070E03010C
:102BB0007A5D01E11200FF0E7B5D01E0B7DA0301EF
:102BC0007B697A6B7D6B120003017A51060A01E181
:102BD000A6D0030A67E0010A5AE0070A45E0010AA5
:102BE00032E0030A28E0010A01E012000401006952
:102BF0000169026903690469056906690769086969
:102C000009690201D26BD36BD46BD56B430E020101
:102C10007A6F7B6B0201000E786F040E796F440EA1
:102C20000201766F776BC1EC18F003017B6F5CDA01
:102C30000301010E7A6F43DA140E64DA01E280D0E8
:102C40000301020E3DD00201D251D311D411D5118E
:102C500035E17BC375F227EC13F0000971E0020146
:102C6000010E70DA030E2CD02ADAC80E4BDA03E319
:102C70000301020E7A6F7BC37EF2B2EC19F00009F9
:102C80005FE064D802085CE10301040E7A6F7BC345
:102C900075F227EC13F0000953E00201030E52DA3B
:102CA000050E0ED07BC37EF2B2EC19F000092FE0C6
:102CB0004DD804010A6F060E0A5D04E10301040EFB
:102CC0007A6F1200050E0A5D29E130DA03017B6993
:102CD0000BDA0301060E7A6FD2C200F2D3C201F200
:102CE000D4C202F2D5C203F2DAC20AF2DBC20BF29C
:102CF000DCC20CF2DDC20DF2D6C20EF2D7C20FF268
:102D0000D8C210F2D9C211F27C817D2B1200D7D922
:102D1000C80EF8D915E30301020E7A6F1200CFD95D
:102D2000640EF0D90DE3CE07000ECF5BD05BD15B14
:102D3000CE51CF11D011D11102E103017A6BD4D958
:102D400012000301080E7A6F96EF18F004010D6B64
:102D500002013C0ECE6FCF6BD06BD16BAAD9020EA5
:102D600004010B5D01E0E2D00C6B0F0E0C5D02E282
:102D7000F7D9FBD70201D20E7F6F020EC0D9D30E56
:102D80007F6F020EBCD9D40E7F6F020EB8D9D50E5C
:102D90007F6F020ED4D904010C6B080E0C5D02E2A9
:102DA000DFD9FBD70C6B060E0C5D0EE282D9040155
:102DB0000C51EA6A040FE96E020EEA22EF500B5D35
:102DC00001E0D6D00C2BEFD70C6B0C510B6E0C6ABC
:102DD0000C50000AE8AE02D0D89004D0CE0E0B5CA6
:102DE000000E0C5802E2BCD9F0D70E6B62D9040178
:102DF0000B51330A62E0CC0A5DE0C90A47E0350AAC
:102E000023E0020A0DE0340A01E07DD052D904012A
:102E10000B0501E0ADD002010D0E7F6F040E48D00E
:102E200089D901E0A5D00201DA0E7F6F020E67D9C1
:102E3000DB0E7F6F020E63D9DC0E7F6F020E5FD94F
:102E4000DD0E7F6F020E34D075D901E291D0020100
:102E5000D60E7F6F020E53D9D70E7F6F020E4FD959
:102E6000D80E7F6F020E4BD9D90E7F6F020E67D935
:102E7000040E04010B5F04010B510B07000952E023
:102E800002010C0E7F6F040E5AD9F5D753D970E1A9
:102E90000201120E7F6F040E32D9110E7F6F040EE5
:102EA0002ED9100E7F6F040E2AD90F0E7F6F040EDD
:102EB00046D938D0010E0E6F35D03CD959E1020108
:102EC000D10E7F6F020E1BD9D00E7F6F020E17D965
:102ED000CF0E7F6F020E13D9CE0E7F6F020E2FD949
:102EE000080ED8800201CE55070ECF55000ED055E2
:102EF000000ED15517E2080ECE5F070ECF5B000E15
:102F0000D05BD15B0FD002010B0E7F6F040E17D97F
:102F100004010B510B07000905E002010C0E7F6F45
:102F2000040EF5D704010E5101E160D7020E0D5DCC
:102F300009E10FC4CAF210C4CBF211C4CCF212C41E
:102F4000CDF211D0CA0EE96E020EEA6EEE500F19E4
:102F500008E1EE50101905E1EE50111902E1EE50B2
:102F6000121901E00D6BE1EC19F004010D51120092
:102F7000E1EC19F0000C0201010EB1D8010EAFD83E
:102F8000060EADD8C7D8120EAAD8230EA8D8340E74
:102F9000A6D8560EDCD8800EDAD8BCD8BBD87D6B4C
:102FA00013EC19F00401196B0C0E195D02E2B7D88D
:102FB000FBD704C27DF213EC19F005C27DF213ECCD
:102FC00019F006C27DF213EC19F007C27DF213EC82
:102FD00019F008C27DF213EC19F009C27DF213EC6E
:102FE00019F00401196B19510B6E0C6A0C50000A90
:102FF000E8AE02D0D89004D0CA0E0B5C000E0C587C
:1030000002E28DD8F0D70201630E69D8820E67D82C
:10301000530E65D8630E63D8350E61D8010E7D6FEF
:1030200013EC19F0E2C27DF213EC19F00201E20593
:1030300018E0D251D311D411D51113E00201360E8C
:103040008AD8CDC27DF213EC19F0CCC27DF213EC1C
:1030500019F0CBC27DF213EC19F0CAC27DF213EC69
:1030600019F00201370E3BD8020E39D8010E37D8BD
:10307000030E7D6F13EC19F0030E0201E25D13E104
:103080000201320E68D8D2C27DF213EC19F0D3C21D
:103090007DF213EC19F0D4C27DF213EC19F0D5C215
:1030A0007DF213EC19F002017D6913EC19F053EF76
:1030B00019F002010B0E7F6F040E9FEF18F05FEC0A
:1030C0002BF00201DE51045C0B6EDF5105580C6ED3
:1030D000E05106580D6EE15107580E6E12007D6FDB
:1030E00013EC19F0020112005FEC2BF004C0DEF2C9
:1030F00005C0DFF206C0E0F207C0E1F212001FD8FF
:10310000020112000B5C000E0C58000E0D58000E50
:103110000E5812007D6B13EC19F00201120002012F
:103120007D6B13EC19F00401192B12007BC37CF2A8
:103130000FEF19F0BEDF040E04010B5D1200806F6B
:10314000BCEF19F0E26F17DFCFDF03011200C7DF1A
:10315000E1DF8AEF18F0C3DF040E7D6F13EF19F083
:08316000A8DF04010C2B120092
:083168000401006B020E005D82
:1031700007E2005169DA00515FDAEF90002BF6D7D1
:1031800012000401490E0C6F020E0D6F0B6B020E44
:103190000B5D44E226DA0C0E5DDAEFCF0CF00D6A1F
:1031A0000E6A0B500C100D100E1032E11ADA0C0ED4
:1031B00076C2EBFF0D0E77C2EBFF02017851791159
:1031C00011E00A0EE66EE66A78C2E6FF79C2E6FF13
:1031D00008DA0CC40BF00DC40CF00CC4E6FF0DC4EF
:1031E000E6FF13DAFED90A0E7AC2EBFF0B0E7BC2A2
:1031F000EBFFF7D90E0EEB6A0F0EEB6AF2D9100E49
:10320000EB6A110EEB6A0BC475F204010B5112004C
:10321000160E0C27000E0D230B2BB9D7FF0C020145
:103220007C5124EF1BF002017551160DF3CF15F4FC
:10323000F4CF16F4490E04011527020E162300DA06
:10324000EE50ED100FE1BED9120EDFC1EBFF1C0EE8
:103250000101FD6FFE6BB6D9DFD9B4D9130EEB6A4D
:10326000140EEB6A7DC2E0F12EEC13F0ABD9130E15
:10327000F1D9EDCF0CF0EE2AEF22E2D9C0D90B5CE8
:103280000E500C5803E3DCD9EE2AEF22D9D9EECF49
:1032900017F4EDCF18F40401D60E175D030E18597C
:1032A00001E301D8010C02017551160DF3CF13F49F
:1032B000F4CF14F4490E04011327020E142387D906
:1032C0000C0E7CD9AFD9F3CF0BF4F4CF0CF47FD92B
:1032D0000A0E74D9A7D9F3CF0DF4F4CF0EF477D931
:1032E0000E0E6CD9EECF0FF4EFCF10F4080E0401E0
:1032F0000F27000E1023116B126B140E0101FD6FCE
:10330000FE6B65D989D90FC451F310C452F3030180
:10331000110E506F5CD913C44EF314C44FF366EC16
:103320001EF00FC45FF310C460F39CEC28F0F3CFE1
:103330000FF4F4CF10F4080E0101E36FE46B010108
:103340000B0EE16F040EE26F37EC13F0DCEC14F0BF
:103350003ED9120E33D9EF683AD90E0EEB6A0F0E32
:10336000EB6A12007EC275F263D9D880EE54000E6B
:10337000ED5401E3000C010C5BD9EE50ED1001E1BE
:10338000000C755159D9EF50010B09E0755154D912
:10339000EF901C0E0101FA6FFB6B34EC15F07AEC28
:1033A00013F07FC2E9FF80C2EAFFEF6E41D9EE065B
:1033B000EF5A755153D9EE50ED1002E1C0EC13F005
:1033C000010C36D9EE50ED1002E0C0EC13F030D90C
:1033D000EE6AED6A1200080E0101E76FE86B010169
:1033E000000EE56F040EE66F81EC13F000C45FF38E
:1033F00001C460F39CEC28F0F3CF00F4F4CF01F4A7
:1034000002C45FF303C460F39CEC28F0F3CF02F432
:10341000F4CF03F404C45FF305C460F39CEC28F01C
:10342000F3CF04F4F4CF05F40401080E045F000E9A
:10343000055B06C45FF307C460F39CEC28F0F3CF90
:1034400006F4F4CF07F481C287F282C288F2020147
:10345000000E856F040E866F12D80401086FFF0EF0
:10346000085D03E1C0EC13F0010C0851F7D804C467
:10347000EEFF05C4EDFF0851DFD8EF80010C040119
:103480000A69490E0B6F020E0C6F096B020E095D83
:103490005BE2A2D80C0E92D8A9D8020E8FD8AFD872
:1034A0000B184BE10E500C1848E196D80A0E86D83E
:1034B0009DD8A5D80B183FE10E500C183CE18CD8D4
:1034C000100E7CD8EECF0FF0EFCF10F0116A126A19
:1034D0000F501010111012102EE187C2E9FF88C2A0
:1034E000EAFF060EB7D8EECF0CF0EECF0DF0EFCF1F
:1034F0000EF072D8060E62D8EE5000010B1908E1EA
:10350000EE500C1905E1EE500D1902E1EE500E19C6
:103510000FE062D8060E52D8E868EE180CE1E868B1
:10352000EE1809E1E868EE1806E1E868EE1803E134
:1035300004010951120009C40AF40401160E0B27F4
:10354000000E0C23092BA2D7FF0E0A5D2AE00A51B8
:10355000160DF3CF0BF4F4CF0CF4490E0B27020E2B
:103560000C230A0EE66EE66A87C2E6FF88C2E6FF13
:1035700033D80BC40BF00CC40CF00BC4E6FF0CC426
:10358000E6FF43D885C2E9FF86C2EAFFEECF0BF023
:10359000EFCF0CF021D80A0E0BC0EBFF0B0E0CC0C6
:1035A000EBFF04010A511200160DF3CFE9FFF4CF2F
:1035B000EAFF490EE926020EEA221200E926000E71
:1035C000EA22120015C4E9FF16C4EAFF120013C470
:1035D000E9FF14C4EAFF12000BC4E9FF0CC4EAFFC0
:1035E00012000CC4E9FF0DC4EAFF1200EECF0BF08D
:1035F000EFCF0CF085C2E9FF86C2EAFF1200EECFE2
:103600000DF0EFCF0EF00D501200D2EC27F0F56E5A
:10361000060EE15EF5501200120EEB500101FC6F38
:1036200047EF15F0EECF5FF3EDCF60F39CEF28F09E
:10363000020175512EEF1BF0B7DF150EDEEF1AF009
:10364000C1DF0E0EDEEF1AF0AFDF0C0EB7DFEE6A51
:10365000ED6A1200B3DFEECF0BF01200A5DF100E03
:04366000DEEF1AF08F
:0C366400150E01019E6F9F6BBCEC00F086
:103670000001816F856BB46B806B140E836F846B5C
:10368000120081C0A4F176EC01F0000907E100010D
:10369000B46B070E876F856B806BB9D081C0B3F1B7
:1036A00029EC03F0000935E038DA0101000EB16FB2
:1036B000040EB26F81C0B0F1EAEC02F000090FE035
:1036C0000001B451B42BEA6A930FE96E000EEA22AE
:1036D00000C4EFFF1F0EB45DE8E1B46BE6D781C014
:1036E000AAF197EC02F00A0E0401005D3FE100012F
:1036F000B451EA6A930FE96E000EEA22EF6AB46BE6
:10370000BED9B5C0CBF0B6C0CCF080D90001876F70
:103710002DD0000185512AE05FEC2BF004C001F4AC
:1037200005C002F406C003F407C004F4C40EE96E39
:10373000000EEA6EEE500401045C016FEE50055875
:10374000026FEE500658036FEE500758046F500E8C
:10375000015D460E0259000E0359000E045906E39E
:10376000DCD90001020E876F010E856F00018551C3
:10377000010A37E0050A04E0040A52E1886BCDD95A
:10378000D7D9FEE0D5D92DE088C0E9FFEA6AE9BEC5
:10379000EA68D890E936EA36950EE926020EEA2262
:1037A000EECF05F4EDCF06F4040105C4F6FF06C420
:1037B000F7FF052B000E06230800F5CF00F4F550A7
:1037C00007E000C4A9F181C0A8F139EC02F0ECD700
:1037D00081C0A6F1BFEC01F000010B0E886F010E55
:1037E000856F070E0001875D1BE087C0CAF019D8FE
:1037F00000090FE00B0E0001885D03E0040E856FE9
:1038000004D0020E875D01E1856B070E876F866B22
:10381000010C0B0E0001885D03E0040E856FB0D72C
:10382000010C0001CA51050A51E0060A4DE0070AE1
:1038300034E0060A30E0030A18E0010A51E1808111
:103840008093010E886F0A0EE66EE66AB7C0E6FF47
:10385000B8C0E6FF890EE66E000EE66E59EC28F061
:10386000F56E060EE15EF550010C80A112D0B7C0D6
:103870003DF2B8C03EF20201890E3B6F000E3C6F74
:10388000B9EC0BF0000904E000018083020E29D09E
:103890000001060E26D073EF1CF0BFC0E6FFC0C0CB
:1038A000E6FF82EC22F0E552E552F3CF84F0C1C08E
:1038B000E6FFC2C0E6FF82EC22F0E552E552F3CF0C
:1038C00083F000010A0E0DD09CEF1CF00A0E886FE9
:1038D000FE0E825D07E082C0A5F17FEC01F0010CD5
:1038E000050E886F010C00018651030A18E0020AD8
:1038F0000FE0010A20E1020E865D02E1E5EC21F015
:10390000FE0E0001825D06E024D90001010E05D003
:1039100015D911E10001030E886F866F000C08D9DC
:103920000AE081C0A4F176EC01F0000904E081C056
:10393000A5F17FEC01F0000C00018651020A32E093
:10394000030A21E0010A61E180B302D0060E5BD0D8
:10395000070E886F83C0A2F184C0A3F18151260DA8
:10396000F3CFE9FFF4CFEAFF000EE926010EEA22C9
:10397000EE52E9CFA0F1EACFA1F1F8EC00F000019E
:10398000826F010E0DD0DAD840E0030137513DE1DE
:1039900010EC22F0F3CFC8F0F4CFC9F00001020E12
:1039A000866F000C82C0B3F129EC03F0000922E01D
:1039B000B4D8C8C041F3C9C042F318EC22F00101E9
:1039C0000B0EB16F040EB26F82C0B0F1EAEC02F0E0
:1039D000000905E00BC443F32EEC22F0F0D748ECCD
:1039E00022F0F3CFC8F0F4CFC9F082C0AAF197EC6F
:1039F00002F0000CA3D809E148EC22F0AAD800019B
:103A0000FE0E826F090E886F010C000C0401076B1B
:103A1000060EE76E0719E8AE02D0E73402D0E75091
:103A2000075D2CE2040EE66EE66A07C4E9FFEA6A67
:103A3000E9BEEA68D890E936EA36890EE926020E30
:103A4000EA22EECF0BF0EFCF0CF00D6A0BC0E6FFD1
:103A50000CC0E6FF0DC0E6FFCBC0E6FFCCC0E6FF22
:103A6000B3EC27F0F56E070EE15EF550000903E1B7
:103A70000401075112000401072BCAD7060C0401E8
:103A80000A6B930E076F000E086F5ED8EF50200888
:103A900004E1072B000E0823F8D707C4B5F008C4CB
:103AA000B6F00001010EC36F4FD8EFCF09F4EF500D
:103AB00033E004010A51010A16E0010A29E1200E4F
:103AC000095D03E02C0E095D05E13ED8EF6A010EA9
:103AD0000A6F1ED00D0E095D03E00A0E095D18E1A4
:103AE00033D8EF6A15D0200E095D12E00001C351F2
:103AF000C32BE96EEA6AD890E936EA36B50EE926B4
:103B0000000EEA2207C4EEFF08C4EDFF04010A6BB1
:103B1000072B000E0823C8D712005FEC2BF004C05F
:103B2000C4F005C0C5F006C0C6F007C0C7F012005B
:103B300081C0A7F124EC02F00009120082C0A4F1B8
:103B400076EC01F00009120007C4E9FF08C4EAFF9F
:0E3B50001200E5EC21F082C0A5F17FEF01F03C
:023B5E00140E43
:103B60000101E76FE86B0101080EE56F040EE66FD7
:103B700081EC13F0F00E04010815400801E0A3D019
:103B80000F0E0815040DF3500B6E0C6A140E0B5E2D
:103B9000000E0C5A0BC01CF40B50140801E293D019
:103BA0001C5100080BE21C510101E76FE86B010199
:103BB0001D0EE56F040EE66F81EC13F012C400F4E5
:103BC00013C401F40401126B136B140E17D9080E01
:103BD000656F040E666FD5EC28F0F3CF04F4F4CFD4
:103BE00005F40401041F051F1C51000810E21C51BC
:103BF00005D91D0E656F040E666FD5EC28F0F3CF66
:103C000006F4F4CF07F40401061F071F02D0066B69
:103C1000076B040EF3D8040E656F040E666FD5ECC7
:103C200028F0F3CF02F4F4CF03F40301080E536F2E
:103C3000040E546FBCD804010251001944E1035131
:103C4000011941E1F00E081540083DE1030146511C
:103C500047110CE046C3E9FF47C3EAFF18C4EEFF73
:103C600019C4EEFF1AC4EEFF1BC4EEFF48C3E9FF00
:103C700049C3EAFF060EE926000EEA2214C4EEFF4D
:103C800015C4EEFF16C4EEFF17C4EEFF4AC3E9FFEA
:103C90004BC3EAFF11C4EFFF04011C510D6E0E6A05
:103CA0000D500A5D0B6E0E500B590C6E140E0B5E10
:103CB000000E0C5A4CC3E9FF4DC3EAFF0BC0EEFFE8
:103CC0000CC0EDFF010CC0EC13F0000C0401450E1C
:103CD0008B6F8C6B140E0301512504018D6F000E48
:103CE0000301522104018E6F0301822B000E8323F6
:103CF00082C38FF483C390F40401916B926B640EC2
:103D0000936F50C394F4956B966B00C297F401C205
:103D100098F402C299F403C29AF44EC3E9FF4FC368
:103D2000EAFF060EE926000EEA22EECF9BF4EECF64
:103D30009CF4EECF9DF4EFCF9EF403018B0E536FF6
:103D4000040E546F34D8140E59D88B0E656F040EC0
:103D5000666FD5EC28F0F3CF95F4F4CF96F4140EFB
:103D6000030151250101F26F000E030152210101EF
:103D7000F36F0101F16B4EC3E9FF4FC3EAFF4EC37E
:103D8000EFF14FC3F0F188EC14F0140E0101E36F72
:103D9000E46B01018B0EE16F040EE26F37EC13F060
:103DA0000B6A0C6A0BC0F3FF0CC0F4FF12002FD893
:103DB000020E15D8020EF3CFEBFF030E24D8040E2B
:103DC0000ED8040EF3CFEBFF050E1DD80A0E07D850
:103DD0000A0EF3CFEBFF0B0E0CC0EBFF1200E9262F
:103DE000000EEA22EECF5FF3EDCF60F39CEC28F0FB
:103DF000F3CF0BF0F4CF0CF007EF1FF00301676F68
:103E0000686B030112000CC0EBFF07EF1FF053C3F8
:083E1000E9FF54C3EAFF1200B0
:083E18001C0E0101E76FE86BCD
:103E20000101000EE56F040EE66F81EC13F0C0ECAB
:103E300013F00301000E706F040E716FF5D80401CA
:103E4000010E001912E1015110E104510B6E0C6AD0
:103E5000060E0B180AE10C5008E105510D6E0E6AB2
:103E6000040E0D1801E10E5001E0000C020E0619BF
:103E700005E1075103E106D9EF6A0DD0010E0619DD
:103E800006E1075104E1010EFDD8EF6E04D0020EE9
:103E9000F9D8EF6E000C020100510401185D2EE10B
:103EA000020101510401195D29E1020102510401DD
:103EB0001A5D24E10201035104011B5D1FE169C386
:103EC000E9FF6AC3EAFF08C4EEFF09C4EEFF0AC4B3
:103ED000EEFF0BC4EEFF0CC4EEFF0DC4EEFF69C392
:103EE000E9FF6AC3EAFF060ED7D80EC4EEFF0FC47F
:103EF000EEFF10C4EEFF11C4EEFF010C000C010E2A
:103F00000401006F016B026B080E036F060E046F55
:103F1000040E056F03016F050BE1010E0401066F2E
:103F2000076B12691369146915691669176914D04A
:103F3000020E0401066F076B6DC3E9FF6EC3EAFF53
:103F4000EECF12F4EECF13F4EECF14F4EECF15F45F
:103F5000EECF16F4EFCF17F404C208F405C209F44B
:103F600006C20AF407C20BF408C20CF409C20DF42D
:103F700000C20EF401C20FF402C210F403C211F425
:103F80007AD8EF500E1902010A151BE174D8010E00
:103F900083D8EF5004010F1902010B1512E16BD801
:103FA000020E7AD8EF500401101902010C1509E134
:103FB00062D8030E71D8EF500401111902010D15DA
:103FC00009E00EC218F40FC219F410C21AF411C29B
:103FD0001BF409D050D8EECF18F4EECF19F4EECF81
:103FE0001AF4EFCF1BF40301000E706F040E716F13
:103FF0001BD81C0E0101F26FF36B0101060EF16F6D
:104000000101120EEF6F040EF06F88EC14F01C0E1D
:104010000101E36FE46B0101000EE16F040EE26F3A
:1040200037EC13F0DCEF14F032D819D8F3CFEEFFF1
:104030000CC0EDFF2CD8020E2FD811D8020EF3CFF2
:10404000EBFF030E0CC0EBFF22D8060E25D807D8D5
:10405000060EF3CFEBFF070E0CC0EBFF1200EECF06
:104060005FF3EDCF60F39CEC28F0F3CF0BF0F4CFCF
:104070000CF047EF20F06DC3E9FF6EC3EAFF060EB8
:104080004CEF20F06BC3E9FF6CC3EAFF120070C372
:10409000E9FF71C3EAFF1200E926000EEA221200CE
:1040A000485454502F312E3020353033200D0A0D16
:1040B0000A5365727669636520556E617661696C35
:1040C00061626C650D0A000D0A0D0A0048545450D7
:1040D0002F312E3020323030204F4B0D0A436F6E7F
:1040E00074656E742D747970653A2000485454508C
:1040F0002F312E3020343034204E6F7420666F758F
:104100006E640D0A0D0A4E6F7420666F756E642E14
:104110000D0A000D0A4E6F772072756E6E696E671C
:10412000206170706C69636174696F6E2E2E2E0051
:104130000D0A526561647920746F20646F776E6C2C
:104140006F6164204D50465320696D616765202D75
:104150002055736520586D6F64656D2070726F74A3
:104160006F636F6C2E0D0A000D0A444843502026E1
:1041700020495020476C65616E696E6720646973E1
:1041800061626C65642E0D0A000D0A44484350209C
:104190002620495020476C65616E696E6720656E08
:1041A00061626C65642E0D0A000D0A4465666175D6
:1041B0006C74205375626E6574204D61736B20289A
:1041C000000D0A44656661756C74204761746577FB
:1041D000617920416464726573732028000D0A447C
:1041E000656661756C742049502041646472657322
:1041F000732028000D0A53657269616C204E756D3D
:10420000626572202800323030206F6B0D0A003258
:104210003236205472616E7366657220436F6D7022
:104220006C6574650D0A0031323520446F6E652E61
:104230000D0A00313530205472616E7366657272FA
:10424000696E6720646174612E2E2E0D0A0035336D
:1042500030204C6F67696E20726571756972656494
:104260000D0A00353032204E6F7420696D706C6518
:104270006D656E7465640D0A00353030200D0A00DE
:10428000323231204279650D0A00323330204C6FD2
:104290006767656420696E0D0A0033333120506111
:1042A0007373776F72642072657175697265640DDE
:1042B0000A003232302052656164790D0A004142B1
:1042C0004F5200504F52540053544F5200515549D1
:0C42D00054005041535300555345520018
:0442DC000301376B38
:1042E000366B03010B0E266F91EC23F0010C0301DA
:1042F00036A103D00B6A0C6A63D0200E0401746FE0
:10430000756B3DC3E9FF3EC3EAFFEF5057E0F5D8B8
:1043100087EC28F0E552E552F3CF3DF3F4CF3EF3BE
:1043200003010F0E336F0301650E316F040E326F00
:1043300074C42FF375C430F30301A00E2E6F31EC5B
:1043400024F0040165512EE1D8D820EC28F0E55284
:10435000E552F3CF76F40401F3500C0802E20C0EA0
:10436000766F7651E66EE66A680EE66E040EE66ECD
:10437000C4D82EEC28F0F56E060EE15EF55000096B
:104380000BE166C43AF367C43BF30301372B66C401
:10439000F3FF67C4F4FF12000F0E04017427000E30
:1043A0007523BED7040E655D09E1661D01E1671D39
:1043B00005E066C474F467C475F4B2D70B680C6882
:1043C0000BC0F3FF0CC0F4FF120003013C6B3691ED
:1043D000375101E0370712003FC338F340C339F3C8
:1043E0003FC32BF340C32CF30301A00E2A6FD2EC82
:1043F00023F0000901E0000C010C71D8030E040148
:10440000655D02E16CD806D0040E655D03E1030131
:104410003869396904016551120026EC24F068D02E
:1044200003013681200E0C6AF36E0CC0F4FF1200FB
:1044300041C338F342C339F341C33CF33F0E030198
:104440003C1741C328F342C329F30301A00E276F91
:104450009CEC23F0000901E0000C010C43C32DF398
:10446000FFEC23F0000901E0000C03013C2B382B8A
:10447000000E3923400E3C5D0AE30AD838C328F306
:1044800039C329F30301A00E276F9CEC23F0010C24
:1044900003013C6B13EC24F00301A00E346F60ECBD
:1044A00024F00009F9E124D03AC33FF33BC340F3C1
:1044B00093DF0401006B016B040100C40BF001C425
:1044C0000CF0002B000E0123030144510B1802E1F4
:1044D00045510C1802E091DFEFD79FDF09D01DECAA
:1044E00024F00401656F0301382B000E39231200FC
:1044F00038C3F3FF39C3F4FF12003DC3E6FF3EC3E8
:04450000E6FF1200C0
:0C450400FF0EE3CFEAFFE552FF0EE3CF0D
:10451000E9FFE552E66AE66AD9CFE6FFDACFE6FFC1
:10452000FC0EE124D96EFF0EE220DA6EE66AE66A3E
:10453000E66A200EEF5C06E0090EEF5C03E0EF6632
:1045400003D03FD0EE50F5D72D0EEF5C03E1FF0E08
:10455000E32A03D02B0EEF5C01E1EE502F0EEF6447
:1045600024D03A0EEF6021D0D890F90EE336FA0E3F
:10457000E336FD0EDECFE3FFFE0EDDCFE3FFD89086
:10458000F90EE336FA0EE336D890F90EE336FA0E5A
:10459000E336FD0EE350DE26FE0EE350DD22300E44
:1045A000EE5CDE26000EDD22D9D7FF0EE3CFE8FF5A
:1045B000E85207E0F90EE31EE32AFA0ED8B4E30648
:1045C000E31EE552E552E552FF0EE3CFDAFFE55276
:1045D000FF0EE3CFD9FFE552E1CFE9FFE2CFEAFFDB
:1045E000ED52ED52EECFF3FFEFCFF4FF1200D9CF33
:1045F000E6FFDACFE6FFFA0EE3CFD9FFFB0EE3CFFB
:10460000DAFFFD0EE35209E72D0EDE6EFC0EE31E0F
:10461000E32AFD0ED8B4E306E31EE652E652E65264
:10462000FD0EE124E76EFF0EE220E46EE652F70E87
:10463000E3CFE6FFF70EE3CFE6FF67EC23F0F90EDA
:10464000E124E96EFF0EE220EA6E57EC23F00AE166
:1046500054EC23F009E157EC23F008E154EC23F08B
:1046600007E108D062EC23F05DEC23F062EC23F06C
:104670005DEC23F062EC23F0DE6AF90EE126FF0E1A
:10468000E222FF0EE3CFDAFFE552FF0EE3CFD9FFC0
:10469000E552FC0EE124E96EFF0EE220EA6EEECF59
:1046A000F3FFEFCFF4FF1200EF380F0B1200EF50C3
:1046B0000F0B02E1EE52D8841200EF380F0B300FCF
:1046C000DE6E1200EE500F0B300FDE6E1200FC0E8D
:1046D000E3CFE9FFFD0EE3CFEAFF100EE66EEE6AD0
:1046E000EE6AEF6AD890FD0EE336FE0EE336ED3645
:1046F000ED36EF36FF0EE30609E088EC23F0EE52CC
:1047000088EC23F0EE5288EC23F0EDD7E56E120032
:10471000030EEF24E8B6EF6E300EEF24E8BEEF6E26
:02472000000C8B
:0E4722003F0EC716C66AC56AC686948694887E
:10473000C68A26C3C8FF120028C3A9F429C3AAF455
:10474000C750040B01E0010EEFD8FAE1C580C5B0F7
:10475000FED7A1B6010C27C335F3EBD801E0010C5D
:10476000C750040B01E0010EDFD8FAE1C5BC19D037
:10477000AAC435F3DED801E0010CC750040B01E0F8
:10478000010ED2D8FAE1A9C435F3D3D801E0010C67
:10479000C750040B01E0010EC7D8FAE1C5AC000C0C
:1047A000020C020C2BC328F32CC329F32AC327F3D2
:1047B000C3DF0401786FE85005E176D80401786F13
:1047C000E85002E078511200C750040B01E0010EDE
:1047D000ABD8FAE1C580C5B0FED7A1B6010C030184
:1047E0002A290301356FA5D801E0010CC750040B3D
:1047F00001E0010E99D8FAE1C5AC000C020CC750DB
:10480000040B01E0010E90D8FAE12DC335F391D8E5
:1048100001E0010CC750040B01E0010E85D8FAE15C
:10482000C5AC000C020CC750040B01E0010E7CD893
:10483000FAE1C584C5B4FED7000C71D8C5B6FED761
:10484000C59AC588C5B8FED7C950120068D8C5B684
:10485000FED7C58AC588C5B8FED7C584C5B4FED7FE
:10486000000C2FC32BF330C32CF32EC32AF39ADF93
:104870000401776FE85016E1030133513307000953
:104880000EE0DBDFE66E030131C3E9FF32C3EAFF6E
:10489000312B000E3223E552E750EF6EEDD7D6DF15
:1048A0000401776F77511200C750040B01E0010E2D
:1048B0003BD8FAE1C584C5B4FED7A1B6010C000C03
:1048C000C750040B01E0010E2FD8FAE1C580C5B036
:1048D000FED7A1B6010C34C335F32BD801E0010C8F
:1048E000C750040B01E0010E1FD8FAE1A1B6010C7C
:1048F000C5BC03D00401A96B03D00401040EA96F49
:10490000C584C5B4FED7A1B6010C0401A95112009B
:1049100035C3C9FFC6BEFF0CC7B0FED7000CC586A5
:10492000C7A0FED7C95012000B6E1F0EC5140B1086
:084930001200EEDF0009120085
:08493800080E0101E76FE86BB6
:104940000101000EE56F040EE66F81EC13F002C466
:104950002EF403C42FF40401026B036B080E030151
:10496000676F686B0301000E656F040E666FD5EC10
:1049700028F0F3CF28F4F4CF29F40401281F291FCD
:10498000080E0B6ED9D8E850EF5ED6D8EF50010173
:10499000E76FE86BE5C2E5F1E6C2E6F181EC13F002
:1049A000CBD8EF500301676F686BE5C265F3E6C2D1
:1049B00066F3D5EC28F0F3CF2AF4F4CF2BF40401FE
:1049C0002A1F2B1F040E0301676F686B0301280E5B
:1049D000656F040E666FD5EC28F0F3CF2CF4F4CF9E
:1049E0002DF40201000EF76F040EF86F7AD8E3C2BF
:1049F000E9FFE4C2EAFF00C4EFFFE9C2E9FFEAC24F
:104A0000EAFF04C4EEFF05C4EDFFEBC2E9FFECC210
:104A1000EAFF06C4EEFF07C4EDFF04012E512C1976
:104A200002E12F512D1901E0000C010C0401016B72
:104A3000EFC200F4026B036BF3C204F4F4C205F49A
:104A4000F5C206F4F6C207F40201F251E66EE66A18
:104A5000F0C2E6FFF1C2E6FF080EE66E040EE66E57
:104A6000D2EC27F0F56E060EE15EF5500201000E65
:104A7000F76F040EF86F35D8080E0201F225030116
:104A8000676F686B000E68230301000E656F040EEC
:104A9000666FD5EC28F0F3CF02F4F4CF03F4080EE0
:104AA0000201F2250301516F526B000E52230301E4
:104AB000010E506FEDC24EF3EEC24FF366EC1EF0E6
:104AC000080E0201F2250101E36FE46B000EE423FE
:104AD0000101000EE16F040EE26F37EC13F0DCEF22
:104AE00014F02FD8040E15D8040EF3CFEBFF050EEB
:104AF0001FD8060E0ED8060EF3CFEBFF070E18D800
:104B0000020E07D8020EF3CFEBFF030E0CC0EBFF33
:104B10001200E926000EEA22EECF5FF3EDCF60F33C
:104B20009CEC28F0F3CF0BF0F4CF0CF0A1EF25F0C4
:104B30000CC0EBFFA1EF25F0E7C2E9FFE8C2EAFFF6
:0C4B40001200F7C2E9FFF8C2EAFF120001
:044B4C000001CD6B2C
:104B5000CE81A0EC12F001EC2AF0B4EC18F088EF52
:104B600000F00401010E3C6F04013C5101E1ECD066
:104B70003C6B0001CD51040A01E1C6D0070A01E1F6
:104B800090D0050A01E17BD0010A6BE0050A38E00C
:104B9000070A2FE0050A02E0010AE6E101013B0EE7
:104BA000ED6F040EEE6F0101CF0EEB6F000EEC6F98
:104BB0000FEC14F000090EE100EC14F00009D4E150
:104BC0000201006B016B026B036B0001CE81D6EC1E
:104BD00015F0CAD70401010E3C6F3B5103E10001FF
:104BE000020E39D0060E3B5D01E08BD00001050EB0
:104BF00032D004013C6B0EEC2AF00009B5E0A1D0E4
:104C00000301D90E4C6F000E4D6F03013B0E4A6F2E
:104C1000040E4B6F0301CF0E486F000E496F030166
:104C2000370E466F040E476FAFEC1DF0000916E01B
:104C30000401010E3C6F3B0503E10001030E0BD0A4
:104C4000060E3B5D03E10001060E05D0110E3B5D33
:104C500004E10001070ECD6F87D73C6BC0EC13F069
:104C600070D0D9C083F2DAC084F20201CF0E816F16
:104C7000000E826FEBEC19F0000910E00DD0D9C0E6
:104C8000B6F1DAC0B7F10101CF0EB46F000EB56F07
:104C900025EC04F0000902E00001CD6B04013C6B3F
:104CA00063D7CD6B290ED880D955000EDA5529E38C
:104CB0000201FD0EEB6F000EEC6F0201FB0EE96FBF
:104CC000000EEA6F0201D90EE76F000EE86F0201D5
:104CD000DB0EE56F000EE66F02013B0EE36F040E84
:104CE000E46F9CEC24F000090AE0080E04013B5D2F
:104CF00006E1010E3C6F0001040ECD6F02D00001F1
:104D0000CD6BC0EC13F030D727EC13F0000901E1B4
:104D10002BD7FDC0F5F2FEC0F6F2FBC0F3F2FCC0EB
:104D2000F4F2D9C0F2F20201DB0EF06F000EF16F67
:104D30000201EF6B0201CF0EED6F000EEE6F16EC6D
:104D400025F00001CD6B10D732EC03F0E4EC15F048
:0C4D500003017CA102D00001CE911200F2
:044D5C004D705374CF
:104D600061636B20322E32302E3034004448435081
:104D70002F476C65616E696E672E2E2E00426F6143
:104D800072642053657475702E2E2E002020202012
:104D900020202020202020202020202000434F4DB4
:104DA0004D414E44532E43474900494E4445582EE9
:104DB00048544D00667470006D6963726F63686972
:104DC00070000D0A0D0A0D4D434850537461636B1A
:104DD0002044656D6F204170706C69636174696F08
:104DE0006E2076312E3120284D70537461636B2014
:104DF000322E32302E30342C205365702032342045
:104E000032303033290D0A0D0A09313A20436861E6
:104E10006E676520426F6172642073657269616CB0
:104E2000206E756D6265722E0D0A09323A20436854
:104E3000616E67652064656661756C7420495020F9
:104E4000616464726573732E0D0A09333A204368F6
:104E5000616E67652064656661756C742067617456
:104E60006577617920616464726573732E0D0A0938
:104E7000343A204368616E67652064656661756CCD
:104E800074207375626E6574206D61736B2E0D0AEC
:104E900009353A20456E61626C65204448435020D4
:104EA0002620495020476C65616E696E672E0D0A99
:104EB00009363A2044697361626C65204448435066
:104EC000202620495020476C65616E696E672E0D63
:104ED0000A09373A20446F776E6C6F6164204D5039
:104EE000465320696D6167652E0D0A09383A2053D3
:104EF000617665202620517569742E0D0A0D0A45CC
:104F00006E7465722061206D656E752063686F69CF
:104F100063652028312D38293A20000D0A496E7624
:104F2000616C696420696E7075742072656365696F
:104F3000766564202D20496E7075742069676E6FE8
:104F40007265642E0D0A507265737320616E79204C
:104F50006B657920746F20636F6E74696E75652E52
:054F60002E2E0D0A00D9
:0A4F6600FB0EE3CFF6FFFC0EE3CFD5
:104F7000F7FFFD0EE3CFF8FFFE0EE3CFE9FFFF0ED4
:104F8000E3CFEAFFF90EE35003E1FA0EE35009E044
:104F9000F90EE30602E2FA0EE3060900F550EE5CB4
:104FA000F1E01200D9CFE6FFDACFE6FFFA0EE3CF49
:104FB000D9FFFB0EE3CFDAFFFC0EE3CFE9FFFD0ED6
:104FC000E3CFEAFFE9CFF3FFEACFF4FFF80EE350B7
:104FD00003E1F90EE35008E0F80EE30602E2F90EF1
:104FE000E306DECFEEFFF2D7FF0EE3CFDAFFE552A6
:104FF000FF0EE3CFD9FFE5521200FB0EE3CFF6FF21
:10500000FC0EE3CFF7FFFD0EE3CFF8FFFE0EE3CF7C
:10501000E9FFFF0EE3CFEAFFE9CFF3FFEACFF4FFAA
:10502000F90EE35003E1FA0EE35009E0F90EE3064E
:1050300002E2FA0EE3060900F5CFEEFFF1D7120007
:10504000FE0EE3CFE9FFFF0EE3CFEAFFF36AF46A57
:10505000EE5203E0F34AF42AFBD71200D9CFE6FF61
:10506000DACFE6FFFA0EE3CFD9FFFB0EE3CFDAFF8C
:10507000FC0EE3CFE9FFFD0EE3CFEAFFF80EE350AD
:1050800003E1F90EE3500AE0F80EE30602E2F90E3E
:10509000E306DE50EF5C02E1EE66F0D7F36EFF0E42
:1050A000E3CFDAFFE552FF0EE3CFD9FFE552F3502D
:1050B0001200D9CFE6FFDACFE6FFFA0EE3CFD9FF31
:1050C000FB0EE3CFDAFFFC0EE3CFE9FFFD0EE3CFEB
:1050D000EAFFE9CFF3FFEACFF4FFF80EE35003E174
:1050E000F90EE3500BE0F80EE30602E2F90EE306D8
:1050F000DECFEFFFEE66F1D7DD52EFD7FF0EE3CF45
:10510000DAFFE552FF0EE3CFD9FFE5521200FE0EA3
:10511000E3CFE9FFFF0EE3CFEAFFE9CFF3FFEACFEA
:10512000F4FF610EEF5C05E67B0EEF5C02E7DF0E3D
:08513000EF16EE52F6E1120049
:0851380060C3F3FF5FC3F4FF45
:105140001200D9CFE6FF61C38CF462C38DF463C350
:105150008EF464C38FF404018C0E906F040E916F73
:1051600090C4E9FFEA6E030EA5D8EF50E66E030E79
:105170009BD88BC4EFFF8FD8020E9CD8010E90D81D
:10518000EF50E66E88D8020E8FD8010E89D88BC4F6
:10519000EFFF8CC404F08DC405F08EC406F08FC4FC
:1051A00007F0E552E7CFD9FF12000401A76BA86B07
:1051B000A96BAA6B67C39FF468C3A0F4D890A0330F
:1051C0009F3365C3A1F466C3A2F49FC40BF0A0C4CF
:1051D0000CF09F07000EA05B0B500C1018E0A1C450
:1051E000E9FFA2C4EAFF020EA127000EA223EECF20
:1051F0000BF0EFCF0CF000010B510401A7270001C9
:105200000C510401A823000EA923AA23DED7030111
:105210006751010B0EE0A1C4E9FFA2C4EAFFEFCF82
:105220000BF000010B510401A727000EA823A923AE
:10523000AA23A9C4A5F4AAC4A6F4A9C49FF4AAC425
:10524000A0F40401A551A6111BE0A96BAA6BA7C489
:105250000BF0A8C40CF00D6A0E6A9FC40FF0A0C436
:1052600010F0116A126A0B500F24A76F0C50102017
:10527000A86F0D501120A96F0E501220AA6FD9D718
:10528000A7C40BF0A8C40CF00B1E0C1E0BC0F3FF40
:105290000CC0F4FF120090C4E9FF91C4EAFF1200B1
:1052A000E926000EEA221200FBDFE552E750EF6E1E
:0E52B0004BEF29F0F5DFEFCF8BF44BEF29F039
:0252BE00F00EF0
:1052C00083160F0E9512959A9598929A839A8398C1
:1052D000809A2EEC0EF0F00E951687D834EC0EF076
:1052E000F00E83D83AEC0EF0F00E7FD80F0E951228
:1052F0000201280E76D8280E74D8080E72D80C0E2B
:1053000070D8010E6ED8130E6CD8800EF96F89EF2D
:1053100029F014D80009FDE1959A9598F00E95169C
:1053200083160201F9390F0B8312839A839852D89E
:10533000F00E83160F0E0201F9155ED0838A839852
:10534000959A95983AEC0EF0808A3AEC0EF083A686
:1053500004D0809A3FD8839A010C809A3BD8839AD4
:10536000000CFAC2E9FFFBC2EAFFEFCF08F4EF50EE
:1053700008E008C4FEF218D80201FA2B000EFB2345
:10538000F0D71200FCC2F6FFFDC2F7FF0800F5CF10
:1053900008F4F55008E008C4FEF206D80201FC2B20
:1053A000000EFD23EFD71200C9DF0009FDE1959A39
:1053B0009598F00E951683160201FE390F0B0F0B10
:1053C00083128388839A06D8F00E83160F0E02018B
:1053D000FE1512D03AEC0EF0808A3AEC0EF0809A6C
:1053E0001200F96F96DF0201120083168382808A11
:1053F0003AEC0EF0809A12008312ECDF0F0E951239
:02540000120098
:0E5402000301156B16691769186919691A6993
:105410001B691C6B1D6B1E6B1F6B1200030115516A
:1054200029E10301260E6B6F040E6C6F03011C0E45
:10543000696F040E6A6F0CEC1FF000092CE0040188
:10544000265115E11CC416F31DC417F31EC418F32E
:105450001FC419F320C41AF321C41BF322C41CF384
:1054600023C41DF324C41EF325C41FF3010C030140
:10547000010E156F27EC13F000090CE003016F6BB0
:1054800003011C0E6D6F040E6E6F7FEC1FF00301A5
:10549000156B010C000C010C20C3E9FF21C3EAFFCE
:1054A000EECF22F4EECF23F4EECF24F4EFCF25F4A9
:1054B0000301010E6F6F03011C0E6D6F040E6E6F02
:1054C0007FEF1FF022C3E9FF23C3EAFF03011C5152
:1054D000EE1808E11D51EE1805E11E51EE1802E12B
:1054E0001F51EE1814E002010E5103011C5D20E172
:1054F00002010F5103011D5D1BE102011051030167
:105500001E5D16E10201115103011F5D11E124C36B
:10551000E9FF25C3EAFF16C3EEFF17C3EEFF18C36A
:10552000EEFF19C3EEFF1AC3EEFF1BC3EEFF010C23
:02553000000C6D
:0E5532005458540048544D0047494600434722
:1055400049004A504700434C41005741560074659A
:1055500078742F706C61696E00000000000000001C
:105560000000746578742F68746D6C000000000092
:10557000000000000000696D6167652F67696600C3
:1055800000000000000000000000746578742F68BF
:10559000746D6C0000000000000000000000696DE8
:1055A0006167652F6A7065670000000000000000F9
:1055B00000006170706C69636174696F6E2F6A615D
:1055C00076612D766D00617564696F2F782D776136
:1055D00076650000000000000000485454502F3150
:1055E0002E3020323030204F4B0D0A436F6E7465E1
:1055F0006E742D747970653A20000D0A0D0A00470B
:0D560000455400494E4445582E48544D0075
:02560E002A0E62
:10561000F66E000EF76E000EF86E03010900F550ED
:105620005A6F0900F5505B6F03E15A6701D03DD016
:105630000900F550556F0900F550566F0900F550F7
:10564000576F09000900F550E96E0900F550EA6E40
:10565000090009000900F550586F0900F550596F0D
:1056600009000900F6CF5CF3F7CF5DF3F8CF5EF3E6
:1056700055C3F6FF56C3F7FF57C3F8FF030158534E
:1056800002E1595307E00900F550EE6E5807F8E2C1
:105690005907F9D75CC3F6FF5DC3F7FF5EC3F8FF98
:0C56A00003015A07000E5B5BBFD712002D
:0456AC003C0ED66E6C
:1056B000D768070ED56ED58EF284F28A1200D9CF44
:1056C000E6FF7EC304F07FC305F080C306F081C30C
:1056D00007F0E552E7CFD9FF1200F2A40AD0D7684D
:1056E0003C0ED66E03017E2B000E7F238023812388
:0456F000F29412001E
:0C56F400FF0EE350136E480E01D04C0E68
:10570000E76EE72EFED7E76AE72EFED7132EF7D710
:045710000000120083
:0C57140015EE00F025EE00F0F86A0A9C8B
:10572000A68EA69C07EC2BF073EC0AF0FDD71200B6
:10573000FF0EE350E84E1200000000D000D000D071
:06574000E82EFAD712006A
:0A5746000000000000F441DD41C145
:0B57500041A9418941684130411341EB
:02575B0000004C
:03575D00EC40CC51
:0557600040C740A0401D
:0B576500D742D242CD42C842C342BE30
:1057700042B2429A428A428042794263424E423366
:075780004227420F420642DE
:0457870000FF00001F
:04578B00000000001A
:020000040030CA
:08000000FFFAFFFEFFFEFBFF0B
:00000001FF
